:060000000C94E9000C94D1
:1000060000000C9400000C9400000C9400000C946A
:1000160000000C9400000C9400000C9400000C945A
:1000260000000C9400000C9483030C94FA030C94C7
:1000360000000C9400000C9400000C9400000C943A
:1000460000000C9418010C9400000C9400000C9411
:1000560000000C9400000C9400000C9400000C941A
:1000660000000C9400000C9400000C9400000301A6
:1000760083010833080000000000000000000000B3
:1000860068010864FA001201000200000020EB0378
:10009600103111030102030105010906A1017501D1
:1000A6009508050719E029E7150025018102950144
:1000B6007508810395057501050819012905910241
:1000C60095017503910395067508150025FF05072B
:1000D600190029FF8100C000040309042603480013
:1000E6005000200049006E0066006F005400650055
:1000F60063006800200053002E0052002E004C00C2
:100106002E00320343006F0064006500560069004C
:10011600730069006F006E00410056005200200017
:100126005500530042002000440065007600690037
:10013600630065000C0330003000300030003100F1
:1001460009022200010100C0320904000001030176
:100156000100092111010001223F00070583030860
:100166000005000100008C0012000200004601227A
:1001760000210000580109002200009E003F0003F4
:100186000000DE000401030904E20026020309045C
:10019600080132030309043A010C1027E80364003E
:1001A6000A0001000010000110000100000000001C
:1001B600000001002D4E414E00494E46000006004B
:1001C6000300B20101008C01B8010000F894EE278B
:1001D600EFBBF1E0F5BFE5BF8DE0A2E0BB27ED93F5
:1001E6008A95E9F780E092E0A0E0B1E0ED9301970F
:1001F600E9F7E4ECF1E085919591009761F0A5911E
:10020600B59105901590BF01F00105900D920197EB
:10021600E1F7FB01F0CFE0E0EEBBEFEFEDBFE2E090
:10022600EEBFC0E8D1E00C943E010A921A92FA920F
:100236006A937A938A939A93AA93BA93EA93FA93D0
:10024600EFB7EA930E940D06E1E0E41528F43A922E
:10025600A62D0E94DD0544244394E991EFBFF99150
:10026600E991B991A9919991899179916991F990B9
:10027600199009901895E0E8E0936100E0E0E093BA
:100286006100E4B9E5B9E0E1E7B9E0E0E8B9EAB967
:10029600EBB9E4BDE5BDE6BDE7BDE8BDE093800092
:1002A600E4E0E09381000E940D06E0E0E093870021
:1002B600E0938600E0938900E0938800E0938B004A
:1002C600E0938A00E0938D00E0938C00E0936E004B
:1002D600E1E0E0936F00A4E7B0E00E942B0278947F
:1002E600E0918201E030E1F3ACEDB5E00E94410619
:1002F6005524E6E05E1660F4449AA4E6B0E00E9457
:1003060041064498A4E6B0E00E9441065394F1CF1A
:100316000E94B301DF01EFEFF0E00E949F063E2E40
:100326000E94B301DF01E2E3F0E00E949F066E2E19
:10033600E9E1E61511F4E1E06E2EEAE1E61511F4C5
:10034600E2E06E2EE9E1E61519F0EAE1E61509F4B8
:1003560001C06624A4E8B3E00E944106D9CFFFCFCE
:10036600E0918C01F0918D0160918E0170918F0169
:10037600ADE6BEE486EC91E40E946C06EE59F848C0
:100386006F4F7F4FE0938C01F0938D0160938E0148
:1003960070938F01FB01FF770895E091ED00E295E0
:1003A600EF70A8E00E944F060895AA930E94C70620
:1003B600ED81FE81E491EF70E1501E2F1F3F09F49D
:1003C60040C0143008F03FC000E0123008F004E0EE
:1003D600E12FF0E0A3E0B0E00E945C06E856FE4F95
:1003E6009F01ED81FE8131961491103051F1113843
:1003F60050F5D901E1E0EC93ED81FE81E491E295BF
:10040600E370E295E07FEE0FEE0FAC81EA2BD901A7
:100416001196EC93113410F010E40DC0113210F067
:1004260010E309C0113110F010E205C0193010F0C8
:1004360010E101C010E0E02FE12BE260D901129635
:10044600EC93E1E001C0E0E00E94CE062796089515
:10045600BA93AA930E94C506E0EAE093D800E0E0CA
:10046600E9BDE6E0E9BDE9B5E0FFFDCFE0E8E093F0
:10047600D800E0E0E093E000E093E100ECE0E093F8
:10048600E2000E941406F098F198E0E0E093820101
:10049600E8E9F1E0FA93EA93E0E0EA93ACE0B0E051
:1004A6000E94FD05EE81FF81309711F4E0E069C0FE
:1004B600EE81FF8172960E94AD06309711F4E0E05E
:1004C60060C0EE81FF817496E491E03011F4E0E0C3
:1004D60058C04E815F8110E01230E8F5FA010491B0
:1004E6000030A9F13596FA93EA93A1E05EDFE03099
:1004F60041F0FA013796FA93EA93A0E056DFE0302E
:1005060011F4E0E03EC0FA0132960E94AD069F016A
:10051600022E032A51F03A932A93E0E0EA93FA0175
:100526003496A491B0E00E94FD05033081F4FA01EF
:100536003196E491E13059F4103011F4F29801C08B
:10054600F29AFA013596E491EF70E0939401475FD1
:100556005F4F1F5FC1CFE0E0E0938B01EDE7E093D3
:100566009501E4EFF1E00E941A06EE81FF8175968F
:10057600A0E8B1E082E00E94B6067E808F80F19A04
:10058600E1E00E94CC06289608950024071408048A
:1005960011F0F19902C0E0E80895E0918201E0309F
:1005A60011F4E1E80895E0E008951A93EEDF1E2FB6
:1005B600E03041F4F8940E941F060E942406E030C1
:1005C60009F410E818C01A93F0DF1E2FE03099F4F2
:1005D6000E941F06E057FE4FE081E27061F0E09155
:1005E600E800E07239F00E941F06E057FE4FA0E0D7
:1005F600A08301C013E8E12F19910895AA930E94E0
:10060600C706E091E9001E2F00918001E091E40009
:100616003E2FE091E800E07229F5EC81EFBF000083
:10062600EFB7EC83F8941093E900E091E400E31748
:1006360079F03091E400015059F40E941F06E0570A
:10064600FE4FA2E0A083E3E80E94CE060C940B06C0
:10065600E0918201E03029F4E1E80E94CE060C9494
:100666000B06D7CFE0E00E94CE060C940B06E09175
:10067600E800E07211F40E9430060E941F06E0575F
:10068600FE4FA1E0A0830895BA93AA930E94C506DF
:100696002FB799DF3E2FE03069F5088519857DDE95
:1006A6004E2FEE81FF81309729F1A22FA7DF3E2F33
:1006B600E03001F5A091F200E42FEA1B5E2FEE81F7
:1006C600FF81A52FB0E0EA17FB0708F45E81E52F4E
:1006D600AE81BF81F0E0AE1BBF0BAE83BF83E52FBB
:1006E6005150E03029F00E943606E093F100F7CF32
:1006F600BEDFD7CF2FBFE32F0E94CC062A960895E0
:100706000A921A928A93AA93BA93EA93FA93EFB744
:10071600EA930E94C7061091E100E0E0E093E10051
:1007260013FF14C0E0E0E093E900E1E0E093EB00A2
:10073600E0E0E093EC00E2E2E093ED00E8E0E09335
:10074600F000E0E0E0938201E0938B0112FF04C029
:10075600E0918201E03009F43DC010E01230B0F4BF
:10076600E12FF0E0E057FE4FE081E17069F0E12F04
:10077600F0E0E057FE4FA0E0A083E12FF0E00E94FA
:1007860024060E94300602C01F5FE8CFE091950163
:10079600E03001F1E0919401E093E900E091E80096
:1007A600E072C1F0A6E9B1E0ED91FD913197FE93BB
:1007B600EE93309779F40E943B0623E831E018E087
:1007C600D9012F5F3F4FEC91E093F1001150C1F733
:1007D6000E9430060E94CE062496E991EFBFF99159
:1007E600E991B991A99189911990099018950A9260
:1007F6001A926A937A938A939A93AA93BA93EA93EC
:10080600FA93EFB7EA932C970E94C506E0E0E093CF
:10081600E900E091E800E87009F4ACC138E0FE01B7
:1008260036968F01E091F100D801EC930F5F1F4FD0
:100836003150C1F7E2EFE093E800AF81A63009F04E
:100846006BC0E72DF82D72960E94AD06E88BF98BEA
:10085600E72DF82D7496249130E03F933F5FE22F09
:10086600AF91AE1708F086C1E889F9890E94B106F2
:10087600E885F9856A857B850E94C00661F4E8896A
:10088600F98934960E94AD06EE87FF87E889F989D3
:100896003696549106C0E889F9893796E88BF98B24
:1008A600DCCF4C85E52FAC85BD85F0E0EA17FB076C
:1008B60008F4452F2091E800E22FE570D9F322FDD8
:1008C6005CC1242F203208F020E2322FEE85FF850E
:1008D600309781F0E32F3150E03059F0EE85FF85F7
:1008E600E491E093F100EE85FF853196EE87FF8770
:1008F600F1CF08C0E32F3150E03021F0E0E0E09383
:10090600F100F8CF421BEEEFE093E800403011F41F
:10091600203209F4CFCF31C1AF81A53061F4EEEFBB
:10092600E093E800E091E800E170E1F3E885E06833
:10093600E093E30022C1AF81A13011F0A33001F5AD
:10094600AE81A230E9F4E885F9853097C9F4EA85E5
:10095600EF772E2F213010F0253008F011C0EEEF82
:10096600E093E8002093E900AF81A33009F402C1C7
:10097600E9E1E093EB00E22FA1E00E944F0628C0D8
:10098600AF81A93019F4AE81A03009F027C0E885FF
:10099600E09382010E941406E0E0E0938B0108E9EF
:1009A60011E0EEEFE093E80031E0353080F430936B
:1009B600E9000E943606E093EB000E943606E093BB
:1009C600EC000E943606E093ED003F5FEECFEEE1CD
:1009D600E093EA00E0E0E093EA00CFC0AF81A83000
:1009E60019F4AE81A03809F00EC002E811E021E04A
:1009F600E091E800E170E1F30E943606E093F10031
:100A06002150D1F71BC0EF81E030E1F420E0AE8148
:100A1600A23859F4EA85E093E900E091EB00E07230
:100A260009F021E0E0E0E093E900E091E800E17000
:100A3600E1F32093F100E0E0E093F100EEEFE093C4
:100A4600E8009BC0AA85BB85129708F093C0EA858B
:100A5600FB85A9E0B0E00E945C06E70DF81DE88B77
:100A6600F98B549131962491AE81A13A61F55330B8
:100A760051F5AF81A130B1F4E889F98932960E9427
:100A8600AD068F01309729F0E889F98934962491CB
:100A9600AFCFE0E0EE87EF874C85ED85E03009F0DB
:100AA6004FEF08CFAF81A33031F4EA85FB85EE56D0
:100AB600FE4F8F019CCFAF81A23029F4213019F46B
:100AC60005E911E094CFAE81A13209F053C053304D
:100AD60009F050C0AF81AB3051F4EEEFE093E8007F
:100AE600EA85FB85EE56FE4FA885A08346C0AF81FA
:100AF600A930A9F5213061F4E091E800E470E1F352
:100B0600E091F100E0938B01EBEFE093E80096CFE4
:100B1600E889F98938964491EC85FD85A42FB0E0E3
:100B2600EA17FB0708F44C85242F203208F020E250
:100B3600E091E800E470E1F3322FE32F3150E0302A
:100B460019F0E091F100F9CF421BEBEFE093E800DA
:100B5600403051F7E091E800E170E1F36FCFAF81EB
:100B6600AA3041F4213031F4E985E09395010E94E1
:100B76003B0664CFE1E2E093EB000E94CC0662966E
:100B8600E991EFBFF991E991B991A991999189916B
:100B960079916991199009901895F29902C0F09887
:100BA60001C0F09AE3E8F1E0FA93EA93A8E0B0E036
:100BB6006BDD0895AA931A93E3E8F1E0FA93EA93BA
:100BC600E0E0EA93A8E0B0E00E94FD05E981E09349
:100BD6008301EA81E0938501E0DF1E2FE03009F012
:100BE60006C0E0E0E0938301E0938501D6DF18813B
:100BF60023960895BA93AA93B981A881109631F0E5
:100C0600FC81EB816A8161931197E9F7EB81FC81A5
:100C160025960895EBE0E0938500ECEDE0938400E3
:100C26000895E0E0E0939001E09391010895E09348
:100C36009601F09397010895E0E0F099E1E0F0E085
:100C46000895A9E0B0E00E945C06E70DF81D359610
:100C5600E491EF70E093E9000895E091E800EE7703
:100C6600E093E8000895D8010F5F1F4FEC910895B7
:100C7600E0919501F0E00E945706D9CF109639F021
:100C860080EA9FE00197F1F7A8951197C9F70895B3
:100C9600F195E195F0400895EE230E2EEA2F19F016
:100CA600EE0F0A94E9F70895EE0FFF1FEE0FFF1FF0
:100CB60008950A2E1B2E81E1AA27BB1B05C010F43E
:100CC600A00DB11DB695A795F795E7958A95B9F745
:100CD60008953F934F935F9351E20A2E1B2E382FB0
:100CE600492FAA27BB278827991B09C020F4A00DE6
:100CF600B11D831F941F96958795B795A7957795F0
:100D06006795F795E7955A9589F75F914F913F91CA
:100D160008950024112490E1AA0FBB1F001C111C8A
:100D26000E1A1F0A18F40E0E1F1E01C0A1609A9516
:100D360099F7FD01D0010895E894B7FF04C0A09586
:100D4600B09511966894F7FDA3DFE3DFFD010EF47D
:100D56009FDF08950590F491E02D0895A591B59132
:100D66008591949108959927EF93FF9305900D929D
:100D76000197E1F7FF91EF910895EA17FB076807DE
:100D8600790708955A934A933A932A931A930A93A2
:100D960008955D814C813B812A81198108810895DE
:00000001FF
